S105001E0001DB
S1048000007B
S123C000C731C713C73AC76EC719C721C729C77CC794C78CC79CC7EEC7E4C7D8C7DDC7F7A7
S123C020C80FC85DC81FC82FC83FC8E5C905C911C925C737CA08C93BC950C945CA64CA7075
S123C040CA7BC96DC959C977C981C991C9D2C9FECA0DCA29CA38CA47C9DEC9EEC9C3C9A9C0
S123C060CA90CA94CA9ACAABCABECAB1CAF4CAC6CB04CB67CB7CCB8ACB9CCB3FCB49CB22CB
S123C080CB52D724D6D0D6FAD712D737D74AD75CD767D77FD7A4D7B4D755D7CFD7E3D7EED8
S123C0A0D7C4D7F9D804D80FD821D82FD83DD6DFD865D88AD875D84BDCB6DD94DD98DDDD43
S111C0C0DA38CB55CB5EDA11DA47DA580000D5
S123C5000101010101CC0000FDFF028EFEFF7F003C8D1A20037EC6BCB680004A26F7CC804F
S123C52001CEC300ED008600A7097EC6BCCE002A4FA700088C003926F8CE10001C260886BB
S123C5403EA7097F00227F0023CC07C0DD261C39801D282086B0A72B860CA72D860597390D
S123C560BDDB2CCC0000DD0CDD12DD148608970BCCC110DD16DD18DD1A8620B7C6A2CEC35C
S123C58000C6208640A7098FC300108F5A26F6CEC300DF08CCC200ED00CCFE00ED04C30063
S123C5A001ED02830100ED06860AA7088620A709EF0CEF0EDC0CC30001DD0CED0ABDDA5808
S123C5C0CEC5E7A6002706BDDAFE0820F6CE10001C200118CE3000180926FC1D20011D0088
S123C5E008CC0000DD2639496E7465726163746976652043202020322E383630206265748D
S123C600610A008D6B8D74816125F881732604863E2068368D513C18388D4C328172270D77
S123C6208177270F816327118162271B39A6008D4A2010188FE700200A188FA400A700EA0D
S123C64000E700863E2034188F373C32331B331B97015D270C8D19A7009B019701085A26BE
S123C660F496018D1620DC8D07368D0416328F39B6102E842027F9B6102F39F6102EC480C3
S123C68027F9B7102F39DE08A608970A1AEE00EE0218E600F7C69B1808FCC000FDC6A0BDC8
S123C6A0FFFF20ED8620B7C6A2DC088FED021AEF00A60981402604EE0CDF0839963C260C83
S123C6C0CE10001F2E2005BDC60320F0120B02ECDE08EE0EDF088CC3002607DC1EC3000162
S123C6E0DD1EA609810026D4BDC686810027CD814027C9812027048602200286048D022033
S123C700BB9701940B910126013996019A0B970B7EC67BEC02A300201CEC02A400E4012030
S123C72014EC02AA00EA01200CEC02A800E8012004EC00E302ED020808398D26A601E60343
S123C7403DDD00A600E6033DDB00D700EC013DDB00D7007D000727064F5F930020D7DC009C
S123C76020D37F00078D6308088D5F090939BDC762EC023CEE0002DF003820D7EC00A30266
S123C7802705CC000020AECC000120A9EC02A3002EF520EEEC02A3002DED20E63CEC002B73
S123C7A01C26043808083937368605B7C7B1EC02380027030926FA380808ED00394F5FA34F
S123C7C00037368604B7C7B120E46D002A094F5FA300ED007300073963006301394F5FA349
S123C7E000ED0039EC002705CC0001ED0039EC0027F64F5FED0039EC02E306DD00E601E9A3
S123C80005A600A904ED04DC00ED06C6043A39EC06A302DD00E605E201A604A20020E6EC3F
S123C82006A302E605E201A604A2002D1E2025EC02A306E601E205A600A2042D0E2015EC92
S123C84006A302260FEC04A3002609C6063ACC0001ED0039C6063ACC0000ED00397F0007BB
S123C860BDC8FB3CC6043ABDC8FBCE0000DF0038A603E6073DDD02A603E6063DD301DD0159
S123C880960089009700A602E6073DD301DD01960089009700A603E6053DD300DD00A6027B
S123C8A0E6063DD300DD00A601E6073DD300DD00EC033DDB00D700A602E6053DDB00D700BA
S123C8C0A601E6063DDB00D700A600E6073DDB00D700C6043ADC02ED02DC00ED007D000732
S123C8E027028D0139CC0000A302DD00C600E2018600A200ED00DC00ED02396D002A058D0B
S123C900E47300073918EC00180818080909ED003918EC020909ED0018EC0018081808189F
S123C92008180820E718E600183A18A60009A70018095A26F518E600183A393CCDEE00E60A
S123C94000384F20C38FCDEE00EE028F0909ED008FCDEE00EE008F20AF18E6003C3AEC00AB
S123C960DD00EC02380909ED00DC00209D18E6003C3AEC003820933CA601CDEE00A7002068
S123C980083CEC00CDEE00ED0018083818080808393CEC00DD00EC02CDEE00ED02DC00ED94
S123C9A00038C6043A57183A39EC00DD00EC02D70718E6003C3AD607ED02DC00ED00380877
S123C9C00820C9EC00D70118E6003C3AD601ED0020B9A6013CEE02273FA70038202AA60184
S123C9E0B7C9EA3CEE0227301C00FF38201AA601B7C9FA3CEE0227201D00FF38200AEC00BB
S123CA003CEE022713ED00380808080839EC00DD00EC023CEE0426063886057EDDE9ED0227
S123CA20DC00ED0038080820DFEC003CEE0227E8E70038ED02080839EC003CEE0227D9ED5F
S123CA400038ED02080839EC00DD00EC023CEE0427C6ED02DC00ED0038EC02ED04DC00EDF8
S123CA60020808393CEE0027AFE6004F38ED00393CEE0027A3EC0038ED00393CEE002798AD
S123CA80EC00DD00EC02380909ED02DC00ED003918EE00391AEE00080839EC00260618EEF2
S123CAA00008083918081808080839EC0026EF20F3EC0027EFCC0001ED0018EE0039EC00A5
S123CAC026E218EE0039EC00DD0018EC00DF04D3048F1AEE002705DC00ED0039DE08864013
S123CAE0A7098621B7C6A2EC0C1AEE0E8FCDEF0C1AEF0E3918EC00DF00D3008F1AEE002793
S123CB00DB080839EC00DD00EC02DD0218EC00DF04D3048F1AEE0227C3DC00ED00DC02ED82
S123CB200239DF00DE08DC00A306CDA300250718081808DE00391809DE0086047EDDE98F1D
S123CB4018E3008F18081808393C323318E3007EC908EE0039EC00DD3A0808180839DC3A3A
S123CB600909ED00180839EC003CEE021AA300382427E302C30002ED02080839EC003CEE09
S123CB80021AA3003824120520E8EC003CEE021AA300382404050520D97EDDE3EC003CEECB
S123CBA0021AA3003824F218A60018083D20C33CBDD640CE00003CDF3DDF3F7F004118300B
S123CBC0CDEE06A600BDCD072528812D260B73004108A600BDCD072519812E260B08A6006E
S123CBE0BDCD0724037ECC753131BDD64A38860F0D39A600BDCD072477BDCC860824F37CEC
S123CC00003DA60008BDCD0725F5812E260AA600BDCD0724030820F681452707816527031B
S123CC207ECCC908A600BDCD072515812D2706812B270520B318630008A600BDCD0724A858
S123CC40803018A70108A600BDCD07241418E601585818EB015880301B18A7010881262282
S123CC608718A601186D002A01409B3D973D2059812E26A408A600BDCD07249C8D0808251B
S123CC808D7A003D20EF963E9743DC3FDD440579003E252C0579003E2526D34436963E9985
S123CCA043973E32251A0579003EDD3F2512E600C0304FD33FDD3F963E89002503973E39F2
S123CCC0DC44DD3F9643973E39CDEF06CE003DBDCD32272C963D18A7018696973DBDCD1331
S123CCE0186D01271B2A0BCECD3DBDD6731860012006CECD41BDD673BDCD51186A0126F858
S123CD003131BDD64A383981302506813922020D390C39CE003D8D1A27147D003E2B0FDC5C
S123CD203F7A003D270A0579003E2AF5DD3F0C390D393736EC002602EC023233393DCCCC64
S123CD40CD41200000BDCFEDBDD640BDCEBCBDD64A7D003D27057D0042260ACC00009741B8
S123CD60DD3DDD3F39964198469741963D9B422A0924168606CEFFFF2009250D8607CE0088
S123CD8000DF40DF3DDF3F0D398B82973DCE00003C3C30BDCDCA6D002B0B69036902690161
S123CDA069007A003D6D032A13A6024CA702260CC601E3002404467C003DED0038DF3E328E
S123CDC09740317D003D27B45F399645D6403DA7019644D6403DE300ED009645D63F3DE337
S123CDE000A70324026C026F006F019643D6403DE302ED029644D63F3DE302ED0224026C80
S123CE00019645D63E3DE302ED0224026C019643D63F3DE301ED0124026C009644D63E3DC0
S123CE20E301ED0124026C009643D63E3DE300ED0039BDD640CED36CBDD6737D0041270389
S123CE40730046BDCEEEBDD64A4FD63DC17F24035F201B53C3FF902F178FDC3E200104099A
S123CE6026FC7D00412A074353C300012A020C3986090D39CC0000DD004FD63DC17F24038B
S123CE805F203353C3FFA02F2F8F96405FDD00DC3E2007047600007600010926F67D004113
S123CEA02A147300007300014353DE0008DF002605C300012A020C3986090D39BDD2D4CE88
S123CEC00045964280972A1BC6038B082A096F00095A26F66F0039C6804A2B035720FAE49D
S123CEE000E7008D028D07964688FF974639963D260EDC42DD3DDC44DD3F964697415F39E4
S123CF007D004227F9D641D84690422510811822ED183C36CE004318CE003E20174081187B
S123CF2022D0183C369642973D96469741CE003E18CE004317363636A8003617A801361738
S123CF40A8023630A606E7061684074CC4185454543AE6034A27095666026601660020F423
S123CF605618A602A900974018A601A901973F18A600A902973E30A6062B15245A76003E4C
S123CF8076003F7600407C003D264CCCCD732053251B73004170004024087C003F26037C48
S123CFA0003E70003F24037C003E70003E7D003E2B252613963D80082326973DDC3F2720D3
S123CFC07F0040DD3E20E67A003D271478004079003F79003E2AF01AEE07C6093A355F3955
S123CFE0CCCD7C1AEE07ED07C6073A35399646984197417D0042260586087ECD757D003D21
S123D00026055F7F004139963D904224052B057ECD7C2B1F8B7E973DDC3E93432B1826063E
S123D020964090452B10DC3E04760040DD3E7C003D26037ECD73DC3EDE43082601090318E9
S123D0403C18DE3EDF3E3CCE00003C3C309645D63F3DA703BDCDF418DF3EDC3FA301DE4323
S123D06003DF3F7F003E383832331838D33EDD3E5F393CCE003DBDCD32260738CC3000ED94
S123D0800039DE3D3CDE3F3C964136BDD640CE00003C3C3C1830CDEE0F86207D004127059F
S123D0A07F0041862DA70008CDEF00CED1DCBDD673BDD1E02E19CED1D8BDD673BDD1E02E3F
S123D0C016186A02CECD41BDD673BDCD5120DC186C02CECD3D20F0CED36CBDD673BDCEEEFF
S123D0E0D63DC07F50CB17200A74003E76003F7600405A26F4860118A70318A6028B082B26
S123D1000A810824064A18A7038602800218A702186D032E15862ECDEE00A70008186D0306
S123D12027058630A70008CDEF00CED1C3860718A705186F04DC3FA301DD3F963EA2009778
S123D1403E2505186C0420EDDC3FE301DD3F963EA900973E18A6048B303CCDEE00A700083E
S123D160186A032605862EA70008CDEF0038080808186A0526BCCDEE0009A600813027F9E8
S123D1800818E602272A8645A70008862BA7005D2A0550862DA70008CDEF004FCE000A023D
S123D1A0378FCB30CDEE00E7000833CB30E700086F00383838BDD64A32974138DF3F38DF78
S123D1C03D38390F42400186A00027100003E800006400000A000001497423FE4B18967FFE
S123D1E096462A12D6412A0EDC421A933D2617DC441A933F20109141260CDC3D1A93422611
S123D20005DC3F1A93440784F424028A080639CE008EC3000026057ECD7C09052AFCDD3E23
S123D2207F00408F9741D73D5F394D2AE24353C30001CEFF8E20DBCE009EC3000026111891
S123D240DE0026037ECD7C0978000179000059492AF5DD3E960097408F9741D73D5F394D58
S123D2602AD57300007300014353DE0008DF002603C30001CEFF9E20C1CE003DBDCD322643
S123D28001397D00412A04860A0D39BDD640860436DE3F3CDE3D3C18308D399642807E4C1B
S123D2A02A03442003448B7E9742BDCFEDBDCEEE7A003D8D1F18EC00DD3D18EC02DD3F1803
S123D2C06A0426E6DC42DD3DDC44DD3F383831BDD64A5F39DC3DDD42DC3FDD44964197461E
S123D2E039BDD640CED43BBDD673BDCFEDBDD64ADC3D1A8385B32B0B7D004126037ECD731C
S123D3007ECD7CBDD6409641367F0041BDCEBCDC4227068086544C26FC5C37CED350BDD631
S123D32000CED34CBDD6732003BDCD51306A0026F832324D2A0CBDD2D4CED594BDD65ABD15
S123D340CFEDBDD64A5F39BDD64020EA402DF8543638EF1D37D00D0139500D013AB60B6180
S123D3603C0888893D2AAAAB3E2AAAAB3F0000003F8000003F800000FFBDD395BDCD517EA1
S123D380D2F08D11BDD640CED43BBDD673BDCD51BDD64A5F3996412704860C0D39963D274F
S123D3A0F8BDD6403C3C30BDD68B4FD63DC07F2A0143BDD22ACED437BDD673BDCD5130BD69
S123D3C0D673BDD68B867F97423C3C30BDD699CED594BDD65ABDCEEE30BDD673BDD68BCE71
S123D3E0D433BDD65ABDCEEE30BDD673BDCFED30BDD68BBDD2D4BDCD51CED416BDD6003006
S123D400BDD673BDCD51383830BDD673BDCEEE3838BDD64A5F393E1D89D93E3A2E8C3E6393
S123D4208E393E9249253ECCCCCD3F2AAAAB40000000FFBF8000003F3172183EDE5BD98634
S123D4400E0D39860D0D39BDD6409641367F0041CED594BDD673BDD1E02F07BDD34786FFBE
S123D46020014F363C3C30BDD68BBDD2D4BDCD51CED49EBDD60030BDD673BDCD5138383278
S123D4804D270CCED49ABDD673730041BDCEEEBDD5EA329741BDD64A5F393FC90FDBBCE20E
S123D4A0DD1B3D70F0F1BD8888893D9D89D9BDBA2E8C3DE38E39BE1249253E4CCCCDBEAA6F
S123D4C0AAAB3F800000FFBDD6404F2005BDD64086F036CED5B2BDD6732003BDCEEE9641A1
S123D4E026F92003BDCEE3BDD1E02EF88D61240930A6002B04880FA7008D54240930A600A2
S123D5002A04880FA7008D47240730A60088F0A700CED5F8BDD673BDCD51BDD2D4BDCD51ED
S123D5203C3C30BDD699A6042A05CED5992003CED584BDD60030A6044724037300414D2BAD
S123D54006BDD673BDCD51383831BDD64A5F397A0042BDD1E02E020C397C0042730041BDFC
S123D560CEEE7A00420D39BDCEBCDC3DDE42DD42DF3DDC3FDE44DD44DF3F9641D6469746E2
S123D580D7415F393638EF1DB9500D013C088889BE2AAAAB3F800000FF37D00D01BAB60B66
S123D5A0613D2AAAABBF0000003F800000FF40490FDB43B40000BDD640BDD2D4BDD4CDBD12
S123D5C0D56ABDD4C7BDCFED2407BDD64A860B0D39BDD64A5F397FFFFFFFBDD640CED5F8F9
S123D5E0BDD673BDCD51BDD64A39BDD640CED5FC20EECED5AE7ED65A3C8EFA3142652EE106
S123D6008FDE3D3CDE3F3C8F9641363CCC0000DD3DDD3FDD40201030A6029746EC03DD44DB
S123D620EC05DD42BDCD5130EE00BDD673BDCEEE38C6043A3CA6004326DD30C6073A353955
S123D640383C3C8F3037367ED699300808BDD67338313131316E00CED5947F0041EC02DD8B
S123D6603FEC00052403730041973D27020D56D73E5F397F0046EC02DD44EC00052403732F
S123D6800046974227020D56D74339DC3FED02DC3D58D1414656ED0039DC44ED02DC4258B4
S123D6A0D1464656ED00397F00415F397D003E2705CC7F80DD3D4F5FDD3F397D003E270381
S123D6C07300415F39BDD67308080808BDD65A393C183CEC00BDD22A183838090920AC3CD7
S123D6E0183C0808BDD65A0909EE00BDD072183838EC00ED0408080808393C183CBDD65A9B
S123D700BDCE7418383824037EDDE9ED00DC00ED02393C183CEC02DD00EC00BDD25F18389D
S123D720387ED68B3C183CBDD65ABDCE4918383824037EDDE9205D3C183CBDD6C5BDCEEEAC
S123D740183838080808087ED68B3C183CBDD6C5BDCEE320EBA6008880A700393C183CBD02
S123D760D6C5BDCD5120093C183CBDD6C5BDCFED18383824037EDDE9080808087ED68B3C77
S123D780183CBDD6C5BDD1E0183838260CCC0001080808080808ED00390808080808086FEF
S123D7A0006F01393C183CBDD6C5BDD1E01838382BDB20E53C183CBDD6C5BDD1E0183838F5
S123D7C02ECB20D53C183CBDD6C5BDD37920A13C183CBDD65ABDD27918383824037EDDE92D
S123D7E07ED68B3C183CBDD65ABDD2F020EA3C183CBDD65ABDD2E120DF3C183CBDD65ABD1A
S123D800D39520D43C183CBDD65ABDD38220C93C183CBDD65ABDD4470736BDD5DA320620DA
S123D820B73C183CBDD65ABDD5EABDD4C720A93C183CBDD65ABDD5EABDD4CD209B3C183C71
S123D840BDD65ABDD5EABDD5B6208D8602E6019D47080839BDDB4BA600BDDC42A601BDDC26
S123D8604208082003BDDB4BA600BDDC42A601BDDC42080839BDDB4B3CEE008602E600275E
S123D880059D470820F738080839183CDF00BDDAA41A830051240C8621B7C6A2DE0018387B
S123D8A0180939DE00DC00C30002E300DD02830002DD04DE02EE000808A60026037ED9FF60
S123D8C0812527037ED9ED08A6008166261BDF02DE0409093CBDD65A380909DF04CEC100A0
S123D8E0BDD072CEC1007ED9DF8164267DDF0218CEC100DE040909DF04EC022A0C862D188A
S123D900A7001808CC0000A302CE000A02378FCE000A02378FCE000A02378FCE000A0237DA
S123D9208FCE000A0237183C388601335D27064FCB30E70008334D27045D27064FCB30E7D4
S123D9400008334D27045D27064FCB30E70008334D27045D27064FCB30E7000833CB30E7CA
S123D96000085FE700CEC10020758178262ADF02DE040909DF04A602BDDC28BDDAEC2572AD
S123D98017BDDAEC256CA603BDDC28BDDAEC256217BDDAEC255C206181632611DF02DE046A
S123D9A00909DF04A603BDDAEC2547204C8162261EDF02DE040909DF04E60318CE0008585C
S123D9C086308900BDDAEC2529180926F2202A8173261ADF02DE040909DF04EE020808A61E
S123D9E0002708BDDAEC250A0820F4200CBDDAEC2409860ABDDAFE2006DE02087ED8B9DE2A
S123DA0000DC00C30002E3008FCC0000ED001838393CDC14C300011A931426FBC30001CE49
S123DA200000081A931426FA8F380909ED00CC000C0909ED007EC73A090909090FDC14EDCD
S123DA4002DC120EED0039EC0008083C183CEE00AD00183838ED00390F3C183CB6103C84A4
S123DA60402605CEFF002003CEBF003CC6C03A18CEE0A31AEF0008083C32324D26F538CC30
S123DA80C500EDFECCDE63EDE2CCDE56EDE0CE10006F226F248600A7211C23181C22181814
S123DAA038380E39960B84082707CC00F0DD062016DC1893162307830001DD062009CC0058
S123DAC0F09316D318DD06960B84102705CC00F02012DC1A931623058300012007CC00F05E
S123DAE09316D31A1A93062302DC06393736BDDAA41A83000224040D323339322001370FE6
S123DB003CDE16088CC2002603CEC110DF16A700960B840827119C18260DDE18088CC2007F
S123DB202603CEC110DF1838330C0E39BDDBC5CC00389D478D2FC60C9D478D298D308D2588
S123DB408601970F8608971C4F971DCC00019D478D13C6069D478D0DC68F9D478D07391897
S123DB60CE011E200418CE0B29180926FC39CC00409D478602CEDB85E6009D478DE1088C88
S123DB80DBC526F439000A1F1F0E04000000001111110F010E00000000000C040800000FBC
S123DBA011110F010E00000C0C000C0C0000000C0C000C0408020006020202120C00000A8B
S123DBC00E04000000CEDBDA18CE0047A60018A7000818088CDC2826F339FF0092CE1000A1
S123DBE00F1D3C201D0010B700946F078104260F8601B710041C0010A6031D0010201E86D9
S123DC0001B710041C0010A6031D001086FFA707B60094A704E7031C00101D00101C3C204F
S123DC20FE00920E3900000036840F8B30813A2B028B071632444444448B30813A2B028B85
S123DC400739BDDC28371686029D47339D4739CE000A02378FCE000A02378FCE000A023765
S123DC608FCE000A02378FCE000A02379D47CC00019D47CC00079D47CC008F9D478602331A
S123DC80CB309D4733CB309D47C62E9D4733CB309D4733CB309D4733CB309D47C66D9D476A
S123DCA0C6739D4739CC00029D478602E60027059D470820F739183CDF00CC7FFFDD04CE56
S123DCC0C3001AEE0E188CC3002607CCE400DD06200518EC04DD06EC0693063CDE00A300E8
S123DCE0382B091A93042E04DF02DD04188CC3002705183C3820CBDC041A837FFF2604865A
S123DD00012015CEC310A609814027158FC300108F8C620026F08602DE00183818097EDD55
S123DD20E93C1838DE02EE0E1AEF0CCDEF0EDE021AEF0ECDEF0CEC0683000118ED04C300AE
S123DD4001DE00A30018ED06A60318A708EC0418ED00860018A709DC0CC30001DD0C18EDE5
S123DD600ADC00E306C30008EE068F09DF0018DF0218EE0436A60018A7003209180983001D
S123DD800126F1DE0218081AEF02DE0009DC0CED00183839862020513CEC00DD00CEC3006A
S123DDA0EC0A1A9300270EEE0E8CC30026F238CC0001ED00399C082604387ECADC183C86F5
S123DDC040A7098621B7C6A2EC0C1AEE0E8FCDEF0C1AEF0E183838CC0000ED00398621B735
S123DDE0C6A2391809860320003CDE084D2602861FA70997018621B7C6A2960181202431DD
S123DE00CEDE33A6002708BDDAEC25F70820F44FD601C00A25034C20F9CB0A8B30BDDAECFF
S123DE2025FB178B30BDDAEC25FB860ABDDAEC25FB38390A52554E54494D4520455252204E
S123DE4000CE1000DC28E316ED161D237FB610008880B710003BCE1000DC26E31EED1E1D48
S123DE6023F73BCE1000CC07D0E31CED1C1D23EFA62236A7220EDE1408DF142605DE1208AC
S123DE80DF127A000A26058621B7C6A286049D47848027037EDF6E9615843F2640960F81B7
S123DEA001223A0F4FC6CF9D47DC1E1A8300642D0BCC0000DD1E961C880C971C961C8408F9
S123DEC02704C6002002C60786029D474FD611C1102502CB30CA809D470E7EDF6E9639846F
S123DEE00126037EDF6E960F8102245EDE1A9C16277C088CC2002603CEC110DF1AE600969F
S123DF000F81002634C10A26068601970F205F9611811F27594C9711811126074F37C6C0EA
S123DF209D4733C120250CC17F2208CEDFB0C0203AE60086029D4720358101260DD710FC94
S123DF40DF9E9D478602970F2024810A2712CEDF9ED60F3AEC009D47960F8B02970F200EE6
S123DF608600970F86019711D610C10A26B5963984042725CE100096224824071C00108B53
S123DF800120031D0010972296234824071C00208B0120031D0020972332B710223B00010E
S123DFA0000600CF020000020011495557777FFF202122232425262728292A2B022D2E2F3B
S123DFC03031323334353637383904053C3D3E3F404142434445464748494A4B4C4D4E4FB9
S123DFE0505152535455565758595A5B5C5D5E5F60616263646566036869066B6C6D6E6FF5
S123E000F0F172737475767778017A7B7C7D7E7F18CE03E8180926FCCE10001F000433CCE8
S123E0201BE61F00042C83000126F7203937368D56CC00029D47CEE05B8602E60027059D50
S123E040470820F732BDDC4232BDDC428602C6299D47CE10001C28204F06CF2A48616C74C8
S123E06065642A2028008D1FCEE077BDDCA5CE10001D23FB8D163B2D504F57455220474CEE
S123E080495443482D20008601979039860E979039CE80004F5FE3008FC300028F8CFF02DD
S107E0A026F4393BEA
S123BFC0E0A3E0A3E0A3E0A3E0A3E0A3E0A3E0A3E0A3E0A3E0A3E0A3E0A3E0A3E0A3E0A32D
S123BFE0DE56DE63E0A3E0A3E0A3E0A3E0A3E010E0A3E0A3E0A3E0A3E0A3E0A3E0A3C500EF
S123FFC0E0A3E0A3E0A3E0A3E0A3E0A3E0A3E0A3E0A3E0A3E0A3E0A3E0A3E0A3E0A3E0A3ED
S123FFE0DE56DE63E0A3E0A3E0A3E0A3E0A3E010E0A3E0A3E0A3E0A3E0A3E0A3E0A3C500AF
S105FF020000F9
S105FF000256A3
S9030000FC
